:020000040000FA
:040000000B303A285F
:08000800A000030EA100831209
:1000100005191028831601178312B23081002B288E
:1000200083160113831203140B190310A80DA90DD5
:10003000AA0DAB0DAC0DAC16FF302C02031D2B2806
:10004000FA302B02031D2B2831152A08AF0029088E
:10005000AE002808AD008B100B11210E8300A00EFE
:04006000200E090065
:0C007400203084008001840A6030040207
:10008000031C3C281230B00009228316FF23900085
:1000900083128316851683120C30851A2C30831632
:1000A000850083128501870107309900003083168F
:1000B00091009F008312C830831681008312313073
:1000C0009000003083168C00831210308B00BC1B14
:1000D0006B28851DA1223C1C6E286D2281018E019A
:1000E0008F010B118B100B108C018B17862031198F
:1000F0008920ED21B30B8428031085190314B90D51
:10010000F030390203197F217622762864003210FC
:10011000080031110130B7008B13203037078316E8
:100120009B001C141A088312A40010303707831692
:100130009B001C141A088312A300A6000230A60616
:100140000030370783169B001C141A088312A20084
:10015000A7000130A7068B17321CB42822090339E7
:10016000A200A309A409A50924082F02031D7929C7
:1001700023082E02031D182922082D02031D7929A8
:1001800001303702031DCB283C19CA283D18CB2863
:100190003D143E14262202303702031DD6283C1996
:1001A000D528BD18D628BD143E142D2203303702A1
:1001B000031DE1283C19E0283D19E1283D153E14B6
:1001C000342204303702031DEC283C19EB28BD19FA
:1001D000EC28BD153E143B2205303702031DF728DD
:1001E0003C19F6283D1AF7283D163E1442220630E7
:1001F0003702031D02293C190129BD1A0229BD1627
:100200003E14432207303702031D0D293C190C29E7
:100210003D1B0D293D173E14442208303702031DB3
:1002200018293C191729BD1B1829BD173E14452252
:1002300026082E02031D792927082D02031D79297E
:1002400001303702031D2B293C192A293D1C2B297B
:100250003D103E14462202303702031D36293C1958
:100260003529BD1C3629BD103E1448220330370203
:10027000031D41293C1940293D1D41293D113E14D2
:100280004A2204303702031D4C293C194B29BD1D5D
:100290004C29BD113E144C2205303702031D57294D
:1002A0003C1956293D1E57293D123E145322063053
:1002B0003702031D62293C196129BD1E6229BD1246
:1002C0003E14542207303702031D6D293C196C2956
:1002D0003D1F6D293D133E14552208303702031D82
:1002E00078293C197729BD1F7829BD133E14562261
:1002F0007929B70A05303702031808008C28013025
:10030000B600B300B400B500B70004308316851AF8
:10031000B700831285018701B1138620B30BBC2976
:10032000031085190314B90DF03039020319E329BC
:10033000B40BBC29013037020319572202303702AF
:1003400003195B220330370203195F22043037029E
:10035000031963220530370203196722063037027A
:10036000031968220730370203196922083037025F
:1003700003196A229630B400311D8D293111321CC7
:10038000C6292D090339AD00AE09AF092F1C8D29EF
:100390008E018F010C1C8D290C102E1E8D298B13A4
:1003A00020303707BB002F08BA00F621103037077E
:1003B000BB002E08BA00F62100303707BB002D081D
:1003C000BA00F6218B1785018701B70AB6010530FF
:1003D0003702031C8D296D2208003E1C08003E10C8
:1003E0001030BB003D08BA00F62108008B133A0814
:1003F00083161C159A003B089B0055309D00AA30BF
:100400009D009C1464009C18022A1C1183128B17F7
:100410000800831600309B001C141A088312BC00CD
:10042000831610309B001C141A0883123C18BD0060
:10043000831620309B001C141A088312C10001305F
:10044000C11BC100C1080319C10008008514400880
:100450004107D0000F08D1000800051440084107EB
:10046000D2000F08D3000800851640084107D400C9
:100470000F08D5000800051640084107D6000F08F0
:10048000D7000800080008000800080085100800D0
:10049000051008008512080005128E018F010C104E
:1004A0004108C0000800080008000800080005080E
:1004B000023A850008000508013A85000800050891
:1004C000203A850008000508103A85000800080059
:1004D000080008000800080008003D188514BD1831
:1004E00005143D198516BD19051608003C1D0800A8
:1004F00050084002031D812A51080F02031C812A63
:10050000851052084002031D8A2A53080F02031C5B
:100510008A2A051054084002031D932A55080F0229
:10052000031C932A851256084002031D9C2A570873
:100530000F02031C9C2A05120C1C08000C10C00A98
:100540000800B601B301B4013C1CA92ABC01BC14CB
:10055000B02ABC1CAE2ABC013C15B02ABC013C141C
:100560003C08B6006400B42AB52AB62AB72AB82ACD
:10057000B41B8514B41F8510B30BB22AB40BB22A76
:100580000310B60CB608031DB22A0030BB003C08AD
:06059000BA00F62108008C
:084000000D00030006000000A2
:02400E00CC01E3
:10420000010078007A007C007E007B0079007F004E
:104210007D007A0078007E007C00FF00FF00FF0038
:104220000000F200F600FA00FE00F200F600FA00CC
:10423000FE00F200F600FA00FE00FF00FF00FF00A3
:10424000010005000500050005000900090009003E
:1042500009000D000D000D000D00FF00FF00FF0024
:10426000FF00FF00FF00FF00FF00FF00FF00FF0056
:10427000FF00FF00FF00FF00FF00FF00FF00FF0046
:10428000FF00FF00FF00FF00FF00FF00FF00FF0036
:10429000FF00FF00FF00FF00FF00FF00FF00FF0026
:1042A000FF00FF00FF00FF00FF00FF00FF00FF0016
:1042B000FF00FF00FF00FF00FF00FF00FF00FF0006
:1042C000FF00FF00FF00FF00FF00FF00FF00FF00F6
:1042D000FF00FF00FF00FF00FF00FF00FF00FF00E6
:1042E000FF00FF00FF00FF00FF00FF00FF00FF00D6
:1042F000FF00FF00FF00FF00FF00FF00FF00DD00E8
:00000001FF
